:020000040000FA
:06000000DD3001303A285A
:08000800A000030EA100831209
:1000100005191028831601178312B23081002B288E
:1000200083160113831203140B190310A80DA90DD5
:10003000AA0DAB0DAC0DAC16FF302C02031D2B2806
:10004000FA302B02031D2B2831152A08AF0029088E
:10005000AE002808AD008B100B11210E8300A00EFE
:04006000200E090065
:0C007400203084008001840A80300402E7
:10008000031C3C281230B000782183160C30850503
:1000900087018312850187010730990000309A009B
:1000A000103083168E008312603083168F00831207
:1000B0000030831691009F008312C83083168100A0
:1000C000831231309000003083168C008312103080
:1000D0008B00402281018E018F010B118B100B10C0
:1000E0008C018B178220311985205A21B30B80286F
:1000F000031085190314B90DF030390203190321D7
:100100000827722864003210080031110130B7004E
:100110008B132030370783169B001C141A08831298
:10012000A4001030370783169B001C141A08831292
:10013000A300A6000230A6060030370783169B00F6
:100140001C141A088312A200A7000130A7068B17FF
:10015000321CB02822090339A200A309A409A50969
:1001600024082F02031DFD2823082E02031DD82872
:1001700022082D02031DFD2801303702031DC3286C
:100180003D143E14802102303702031DCA28BD14DD
:100190003E149B2103303702031DD1283D153E1428
:1001A000B62104303702031DD828BD153E14D121D5
:1001B00026082E02031DFD2827082D02031DFD28F9
:1001C00001303702031DE7283D103E14EC210230B8
:1001D0003702031DEE28BD103E1401220330370202
:1001E000031DF5283D113E14162204303702031D6D
:1001F000FC28BD113E142B22FD28B70A053037021A
:100200000318080088280130B600B300B400B50018
:10021000B70085018701B1138220B30B2929031090
:1002200085190314B90DF030390203195029B41F90
:100230008501B41F8701B40B29293708B6080319B3
:10024000B60003192729FF3085008700B6039630D2
:10025000B400311D0C293111321C33292D09033909
:10026000AD00AE09AF092F1C0C298E018F010C1CAB
:100270000C290C102E1E0C298B1320303707BB00C5
:100280002F08BA00632110303707BB002E08BA00D0
:10029000632100303707BB002D08BA0063218B179C
:1002A00085018701B70AB60105303702031C0C2906
:1002B000402208003E1C08003E101030BB003D08E4
:1002C000BA00632108008B133A0883161C159A00A4
:1002D00083123B0883169B0055309D00AA309D0079
:1002E0009C1464009C1871291C1183128B17080040
:1002F000831610309B001C141A088312BD000800DE
:100300003D146430DC00CD22E0006730DC00CD22FB
:10031000E1006530DC00CD22C4006630DC00CD2277
:10032000CC006830DC00CD22D0000130C800D40001
:10033000FF30C0000800BD146430DC00D722E200AA
:100340006730DC00D722E3006530DC00D722C5002F
:100350006630DC00D722CD006830DC00D722D10027
:100360000130C900D500FF30C10008003D156430E0
:10037000DC00E122E4006730DC00E122E5006530CA
:10038000DC00E122C6006630DC00E122CE006830ED
:10039000DC00E122D2000130CA00D600FF30C200EA
:1003A0000800BD156430DC00EB22E6006730DC009D
:1003B000EB22E7006530DC00EB22C7006630DC0092
:1003C000EB22CF006830DC00EB22D3000130CB0001
:1003D000D700FF30C3000800601A0512E01A85122A
:1003E000601B0510E01B851061188710E1180711CC
:1003F00061190710E1198712611A0712E11A8711B2
:100400000800621A0512E21A8512621B0510E21B2F
:10041000851063188710E318071163190710E31993
:100420008712631A0712E31A87110800641A05126B
:10043000E41A8512641B0510E41B851065188710EB
:10044000E518071165190710E5198712651A0712D3
:10045000E51A87110800661A0512E61A8512661B4E
:100460000510E61B851067188710E7180711671934
:100470000710E7198712671A0712E71A8711080091
:100480003D188021601C3D10BD189B21621CBD10D1
:100490003D19B621641C3D11BD19D121661CBD1149
:0204A000080052
:10052000681E962A5A1C05125A180516E81E9C2A9F
:10053000DA1C8512DA188516681FA22A5A1D0510C2
:100540005A190514E81FA82ADA1D8510DA1985142E
:10055000691CAE2A5B1C87105B188714E91CB42A3F
:10056000DB1C0711DB180715691DBA2A5B1D071074
:100570005B190714E91DC02ADB1D8712DB198716DA
:10058000691EC62A5B1E07125B1A0716E91ECC2AD3
:10059000DB1E8711DB1A8715080003308A00DC1385
:1005A0005C08820003308A00DC175C08820004309B
:1005B0008A00DC135C08820004308A00DC175C08C7
:1005C000820005308A00DC135C08820005308A0056
:1005D000DC175C08820006308A00DC135C088200AD
:0A05E00006308A00DC175C08820078
:10060000003401340234033404340534063407342E
:10061000083409340A340B340C340D340E340F34DE
:10062000103411341234133414341534163417348E
:10063000183419341A341B341C341D341E341F343E
:1006400020342134223423342434253426342734EE
:10065000283429342A342B342C342D342E342F349E
:10066000303431343234333434343534363437344E
:10067000383439343A343B343C343D343E343F34FE
:1006800040344134423443344434453446344734AE
:10069000483449344A344B344C344D344E344F345E
:1006A000503451345234533454345534563457340E
:1006B000583459345A345B345C345D345E345F34BE
:1006C0006034613462346334F13464341E343F3452
:1006D0000134003400340034003400340034003479
:1006E000003400340034003400340034003400346A
:1006F000003400340034003400340034003400345A
:10070000003401340234033404340534063407342D
:10071000083409340A340B340C340D340E340F34DD
:10072000103411341234133414341534163417348D
:10073000183419341A341B341C341D341E341F343D
:1007400020342134223423342434253426342734ED
:10075000283429342A342B342C342D342E342F349D
:10076000303431343234333434343534363437344D
:10077000383439343A343B343C343D343E343F34FD
:1007800040344134423443344434453446344734AD
:10079000483449344A344B344C344D344E344F345D
:1007A000503451345234533454345534563457340D
:1007B000583459345A345B345C345D345E345F34BD
:1007C0006034613462346334003400340034003403
:1007D0000034003400340034003400340034003479
:1007E0000034003400340034003400340034003469
:1007F0000034003400340034003400340034003459
:10080000003401340234033404340534063407342C
:10081000083409340A340B340C340D340E340F34DC
:10082000103411341234133414341534163417348C
:10083000183419341A341B341C341D341E341F343C
:1008400020342134223423342434253426342734EC
:10085000283429342A342B342C342D342E342F349C
:10086000303431343234333434343534363437344C
:10087000383439343A343B343C343D343E343F34FC
:1008800040344134423443344434453446344734AC
:10089000483449344A344B344C344D344E344F345C
:1008A000503451345234533454345534563457340C
:1008B000583459345A345B345C345D345E345F34BC
:1008C0006034613462346334F13464341E343F3450
:1008D0000134003400340034003400340034003477
:1008E0000034003400340034003400340034003468
:1008F0000034003400340034003400340034003458
:10090000003401340234033404340534063407342B
:10091000083409340A340B340C340D340E340F34DB
:10092000103411341234133414341534163417348B
:10093000183419341A341B341C341D341E341F343B
:1009400020342134223423342434253426342734EB
:10095000283429342A342B342C342D342E342F349B
:10096000303431343234333434343534363437344B
:10097000383439343A343B343C343D343E343F34FB
:1009800040344134423443344434453446344734AB
:10099000483449344A344B344C344D344E344F345B
:1009A000503451345234533454345534563457340B
:1009B000583459345A345B345C345D345E345F34BB
:1009C0006034613462346334003400340034003401
:1009D0000034003400340034003400340034003477
:1009E0000034003400340034003400340034003467
:1009F0000034003400340034003400340034003457
:100A0000003401340234033404340534063407342A
:100A1000083409340A340B340C340D340E340F34DA
:100A2000103411341234133414341534163417348A
:100A3000183419341A341B341C341D341E341F343A
:100A400020342134223423342434253426342734EA
:100A5000283429342A342B342C342D342E342F349A
:100A6000303431343234333434343534363437344A
:100A7000383439343A343B343C343D343E343F34FA
:100A800040344134423443344434453446344734AA
:100A9000483449344A344B344C344D344E344F345A
:100AA000503451345234533454345534563457340A
:100AB000583459345A345B345C345D345E345F34BA
:100AC0006034613462346334F13464341E343F344E
:100AD0000134003400340034003400340034003475
:100AE0000034003400340034003400340034003466
:100AF0000034003400340034003400340034003456
:100B00000034013402340334043405340634073429
:100B1000083409340A340B340C340D340E340F34D9
:100B20001034113412341334143415341634173489
:100B3000183419341A341B341C341D341E341F3439
:100B400020342134223423342434253426342734E9
:100B5000283429342A342B342C342D342E342F3499
:100B60003034313432343334343435343634373449
:100B7000383439343A343B343C343D343E343F34F9
:100B800040344134423443344434453446344734A9
:100B9000483449344A344B344C344D344E344F3459
:100BA0005034513452345334543455345634573409
:100BB000583459345A345B345C345D345E345F34B9
:100BC00060346134623463340034003400340034FF
:100BD0000034003400340034003400340034003475
:100BE0000034003400340034003400340034003465
:100BF0000034003400340034003400340034003455
:100C00000034013402340334043405340634073428
:100C1000083409340A340B340C340D340E340F34D8
:100C20001034113412341334143415341634173488
:100C3000183419341A341B341C341D341E341F3438
:100C400020342134223423342434253426342734E8
:100C5000283429342A342B342C342D342E342F3498
:100C60003034313432343334343435343634373448
:100C7000383439343A343B343C343D343E343F34F8
:100C800040344134423443344434453446344734A8
:100C9000483449344A344B344C344D344E344F3458
:100CA0005034513452345334543455345634573408
:100CB000583459345A345B345C345D345E345F34B8
:100CC0006034613462346334F13464341E343F344C
:100CD0000134003400340034003400340034003473
:100CE0000034003400340034003400340034003464
:100CF0000034003400340034003400340034003454
:100D00000034013402340334043405340634073427
:100D1000083409340A340B340C340D340E340F34D7
:100D20001034113412341334143415341634173487
:100D3000183419341A341B341C341D341E341F3437
:100D400020342134223423342434253426342734E7
:100D5000283429342A342B342C342D342E342F3497
:100D60003034313432343334343435343634373447
:100D7000383439343A343B343C343D343E343F34F7
:100D800040344134423443344434453446344734A7
:100D9000483449344A344B344C344D344E344F3457
:100DA0005034513452345334543455345634573407
:100DB000583459345A345B345C345D345E345F34B7
:100DC00060346134623463340034003400340034FD
:100DD0000034003400340034003400340034003473
:100DE0000034003400340034003400340034003463
:100DF0000034003400340034003400340034003453
:100E1000DA01DA1B80215A1B9B21DA1AB6215A1AF1
:100E2000D1210A300F02031C08008E018F013D1CE6
:100E3000382FC80B382FD40B382F4C08C800500857
:100E4000D400C00A440840020318342F4008DC00D4
:100E5000CD22DA004008DC00D222DB006008E80086
:100E60006108E9009022382FC0016018262F3D103C
:100E7000BD1C592FC90B592FD50B592F4D08C9002F
:100E80005108D500C10A450841020318552F4108F1
:100E9000DC00D722DA004108DC00DC22DB0062083B
:100EA000E8006308E9009022592FC1016218472F1A
:100EB000BD103D1D7A2FCA0B7A2FD60B7A2F4E0804
:100EC000CA005208D600C20A460842020318762F0A
:100ED0004208DC00E122DA004208DC00E622DB0006
:100EE0006408E8006508E90090227A2FC2016418BE
:100EF000682F3D11BD1D9B2FCB0B9B2FD70B9B2F1D
:100F00004F08CB005308D700C30A47084302031811
:100F1000972F4308DC00EB22DA004308DC00F022C4
:100F2000DB006608E8006708E90090229B2FC301F8
:080F30006618892FBD110800AD
:084000000F00030006000000A0
:02400E00CC33B1
:10420000010078007A007C007E007B0079007F004E
:104210007D007A0078007E007C00FF00FF00FF0038
:104220000000F200F600FA00FE00F200F600FA00CC
:10423000FE00F200F600FA00FE00FF00FF00FF00A3
:10424000010005000500050005000900090009003E
:1042500009000D000D000D000D00FF00FF00FF0024
:10426000FF00FF00FF00FF00FF00FF00FF00FF0056
:10427000FF00FF00FF00FF00FF00FF00FF00FF0046
:10428000FF00FF00FF00FF00FF00FF00FF00FF0036
:10429000FF00FF00FF00FF00FF00FF00FF00FF0026
:1042A000FF00FF00FF00FF00FF00FF00FF00FF0016
:1042B000FF00FF00FF00FF00FF00FF00FF00FF0006
:1042C000FF00FF00FF00FF00FF00FF00FF00FF00F6
:1042D000FF00FF00FF00FF00FF00FF00FF00FF00E6
:1042E000FF00FF00FF00FF00FF00FF00FF00FF00D6
:1042F000FF00FF00FF00FF00FF00FF00FF00DD00E8
:00000001FF
